:100000000000000000003328FF0003088301FE0009
:100010000408FD00852883169B0083169C011C1490
:100020001A089B0A2F2883178001840AFF3E031DAC
:1000300014282F28A501E83EA400A509FC30031CC4
:100040002428A40703182128A4070000A50F2128AD
:1000500024182A28A41C2E2800002E280800831308
:10006000831203130800830107309F008330831637
:10007000810060308B008C0183128C010B30831661
:100080008E0083129001920107309F009701980122
:10009000831698010C3099009201203084005D3065
:1000A00083121420A03084005030142020308400AB
:1000B00030301320DF3083168500831285012B300A
:1000C0008316860083128601903098008430831650
:1000D000980083128C1283168C16831231272D30D0
:1000E000E700E8006330D200FA30FC00AF1781016E
:1000F0000B118B1764302A0203188428C330A50023
:1001000050301B20AA0A7A282C29000064008C1E7B
:100110009F288C121A08F50002302E02031C9C281E
:1001200028302E0203189C28A03084002E08840753
:1001300002308402750880000C30D400AE0A0B1D1A
:1001400021290B110612CF080319A828CF03061680
:10015000D4080319B428D403D408031DB428AE016D
:10016000AF140530CD002F10F60A19307602031CAB
:10017000F228F6012F158617203052020318C528E1
:100180004E0C03188617031C8613CE080319C928C2
:10019000CE03CC080319DB28CC03CC08031DDB28D5
:1001A000AE01D4010530CD002F100D304B02031DE0
:1001B000DB280C30CB00CC08031DE628CD08031942
:1001C000E628CD03CD08031DE6282F14D008031917
:1001D000EF28D0038316061083120610F128831629
:1001E00006148312F70AF5307702031C1B29F70166
:1001F000C9080319FD280330CF00861D0129E1300D
:10020000CF00790A031D0629FF30CF00AF1D0A2950
:100210007D30CF00F00803190E29F003F10803190F
:100220001229F103EF0803191629EF03F208031945
:100230001A29F203F80A0A307802031C2129F8016E
:10024000AF167D0884007E088300FF0E7F0E090034
:100250006430D000C830CC00B001D801D701D9013A
:10026000CB010530CD002F1008304B0203183A297E
:100270006330D2002F1D3D2A0B300B20AD0003014F
:10028000051B013E2D18013C031D492900300B20A0
:10029000E9000301851B013EAD18013C031D5329F4
:1002A00001300B20EA0003010518013E2D19013C25
:1002B000031D5D2902300B20EB0003018518013E70
:1002C000AD19013C031D672903300B20EC0003012D
:1002D0000519013E2D1A013C031D712904300B2024
:1002E000ED0003018519013EAD1A013C031D7B2978
:1002F00005300B20EE008619802908300B20EF0016
:10030000861E84290A30F2003F30C900E90803192B
:100310008B29E9034910EA0803199029EA03C91057
:10032000EB0803199529EB034911EC0803199A29E5
:10033000EC03C911ED0803199F29ED034912EE08DA
:100340000319A429EE03C9120C300B20AD004F3065
:10035000E100EF080319B1292D08F9006630E0002B
:10036000B529FF30F9004E30E0004F30E300F208CD
:100370000319BE292F174E30E200C1292F13663012
:10038000E200791CCB29491CCB294A18CB292F160E
:100390004A143130DA00F91CD529C91CD529CA18EC
:1003A000D5292F16CA143130DB00791DDF29491DEC
:1003B000DF294A19DF292F164A153130DC00F91DD3
:1003C000E929C91DE929CA19E9292F16CA153130A9
:1003D000DD00791EF329491EF3294A1AF3292F1645
:1003E0004A163130DE00F91EFD29C91EFD29CA1A40
:1003F000FD292F16CA163130DF002F1E0C2A2F12AE
:10040000D508031D062A09300B20F0000D300B2003
:10041000D5000A300B20F1007A08790203191B2A53
:100420007908FA00F0010E300B20D500FF30790278
:1004300003181B2AF1010301AF1B013E2F1B013CD6
:100440000319292AAF172F1FAF13F0010E300B200D
:10045000D500F10803192F2A0617AF15372A0613FE
:10046000AF114908CA00D508031D372A3127FC08F7
:1004700003193C2AFC03D5012F11AF1E522AD508BF
:10048000031D522A4A27CC30AD005A27BE30AD009A
:100490005A277D274A27CC30AD005A274430AD007B
:1004A0005A27AF122F1CDF2CB00ACB08031D672A76
:1004B00041308316A0005430A1004530A2003030F6
:1004C000A3000D30A40005308312D300B62C0130F8
:1004D0004B02031D7A2A41308316A0005430A1003C
:1004E0005630A2003130A3000D30A4000530831235
:1004F000D300B62C02304B02031D962A41308316DE
:10050000A0005430A1002B30A2004330A3004D3096
:10051000A4004530A500A6003D30A7003130A8005A
:100520000D30A9000A308312D300B62C03304B02E1
:10053000031DB32A41308316A0005430A1002B3094
:10054000A2004330A3004D30A4004730A500463040
:10055000A6003D30A7003130A8000D30A9000A30B8
:100560008312D300B62C04304B02031DD82A41302D
:100570008316A0005430A1002B30A2004330A3000A
:100580005330A4004330A5005330A6003D30A700EF
:100590002230A8004730A9005330AA004D30AB00EC
:1005A0002230AC000D30AD000E308312D300B62CDB
:1005B00005304B02031DF92A41308316A000543048
:1005C000A1002B30A2004330A3004E30A4004D30D8
:1005D000A5004930A6003D30A7003230A8002C30DD
:1005E000A9003230AA000D30AB000C308312D300CA
:1005F000B62C06304B02031D162B41308316A0008B
:100600005430A1002B30A2004330A3005330A4008B
:100610004330A5004230A6003D30A7003130A8008D
:100620000D30A9000A308312D300B62C07304B02DC
:10063000031D332B41308316A0005430A1002B3012
:10064000A2004330A3004C30A4004930A500503034
:10065000A6003D30A7003130A8000D30A9000A30B7
:100660008312D300B62C08304B02031D502B4130AF
:100670008316A0005430A1002B30A2004330A30009
:100680004D30A4004730A5004430A6003D30A700FF
:100690003430A8000D30A9000A308312D300B62CE4
:1006A00009304B02031D6B2B41308316A0005430E0
:1006B000A1002B30A2004330A3005230A4004530EB
:1006C000A5004730A6003F30A7000D30A800093034
:1006D0008312D300B62C0A304B02031D822B41300B
:1006E0008316A0005430A1002B30A2004330A30099
:1006F0005330A4005130A5000D30A60007308312FE
:10070000D300B62C0B304B02031D932B41308316C4
:10071000A0005430A1004830A2000D30A3000430E6
:100720008312D300B62C0C304B02031DE32B413057
:100730008316A0005430A1002B30A2004330A30048
:100740004D30A4004730A5005330A6003D30A7002F
:100750002230A8002B30A9003330AA0083123108C0
:100760008316AB00831232088316AC008312330861
:100770008316AD00831234088316AE008312350849
:100780008316AF00831236088316B0008312370831
:100790008316B100831238088316B2008312390819
:1007A0008316B30083123A088316B40083123B0801
:1007B0008316B5002230B6000D30B7001830831212
:1007C000D300D90AB62C0D304B02031DB62C433092
:1007D0008316A0004830A1005F30A2003130A30092
:1007E0003A30A4002030A50083125A088316A600D0
:1007F0000A30A7004330A8004830A9005F30AA00A3
:100800003230AB003A30AC002030AD0083125B08D0
:100810008316AE000A30AF004330B0004830B1005C
:100820005F30B2003330B3003A30B4002030B5004E
:1008300083125C088316B6000A30B7004330B80054
:100840004830B9005F30BA003430BB003A30BC00E9
:100850002030BD0083125D088316BE000A30BF0041
:100860004330C0004830C1005F30C2003530C300A3
:100870003A30C4002030C50083125E088316C600DB
:100880000A30C7004330C8004830C9005F30CA0092
:100890003630CB003A30CC002030CD0083125F08D8
:1008A0008316CE000A30CF0030308312D3000127E8
:1008B00053308316A0006530A1006330A2003A30A7
:1008C000A3002030A400831261088316A5008312C0
:1008D00060088316A6000A30A7005030A8006F30C9
:1008E000A9007730AA003A30AB002030AC00831268
:1008F00063088316AD00831262088316AE000A30C7
:10090000AF005430B0006D30B1007030B2003A30FA
:10091000B3002030B400831264088316B50083123C
:1009200065088316B600831266088316B700203068
:10093000B8004330B9000A30BA004730BB0073300A
:10094000BC006D30BD003A30BE002030BF008312C5
:1009500067088316C000831268088316C1001A3026
:10096000C2000D30C30024308312D3000E304B027E
:100970000318BB2C012708304B02031CC72C09307D
:100980004B020319C72C0A304B02031DCA2C1E3020
:10099000CC00DC2C08304B020319DA2C0B304B0254
:1009A0000319DA2C0C304B020319DA2C0D304B02F0
:1009B000031DDC2CFA30CC000530CD002F10AF1C0D
:1009C000A62EAF1009304B02031CEA2C0B304B0251
:1009D000031DFE2C831620088312A3004F30230230
:1009E000031DFD2C831621088312A3004B30230224
:1009F000031DFD2CCC01CB0AB001A62E09304B0201
:100A00000319062D0A304B02031D402E83162008C1
:100A10008312A3002B302302031D462D83162108C9
:100A20008312A30043302302031D462D83162208A0
:100A30008312A30052302302031D462D8316230880
:100A40008312A30045302302031D462D831624087C
:100A50008312A30047302302031D462DCC01D80A80
:100A6000831629088312A3003130230203193C2D79
:100A700035302302031D402DD8010A30CB00422D12
:100A80006330D200B0013230CD002F108316200821
:100A90008312A3002B302302031DA72D83162108E8
:100AA0008312A30043302302031DA72D83162208BF
:100AB0008312A30053302302031DA72D831623089E
:100AC0008312A30051302302031DA72DCC0109304E
:100AD000CB00831626088312A30030302302AA001D
:100AE000AD01831626088312E7002030E800831644
:100AF00027088312A3002C3023020319962D831696
:100B000027088312E80003102A0DAD000310AD0D75
:100B10000310AD0D2A08AD072A082D07AA00831679
:100B200027088312A30030302302AD002D082A07C6
:100B3000D200D70A203052020318A62DD701CE08C2
:100B4000031DA62D0310520CCE00CE0AB001831651
:100B500020088312A30052302302031D1B2E83168C
:100B600021088312A30049302302031D1B2E831684
:100B700022088312A3004E302302031D1B2E83166E
:100B800023088312A30047302302031D1B2ECC0130
:100B9000FF30D6000430AA0012302A020318172EA4
:100BA0002A08A03E84000008A30022302302031D6F
:100BB000132E2A0AA03E84000008A300333023022B
:100BC000031D132EAB010B302B020318FA2D02303C
:100BD0002A07AC002B08AC072C08A03E84000008B4
:100BE000AD002B083D3E84002D0880000130AB078E
:100BF000031CE32D0F30D100AC010A302C02031886
:100C0000092ED526E8260B30D1070130AC07031C8E
:100C1000FD2DFF3056020318122E5608D100D5269E
:100C20000B30CB00172E0130AA07031CCC2DB001CE
:100C30000530CD002F10831620088312A3002B301F
:100C40002302031D3F2E831621088312A300433085
:100C50002302031D3F2E831622088312A3004D306A
:100C60002302031D3F2E831623088312A300543052
:100C70002302031D3F2ECC010830CB00B001A62E6D
:100C80000C304B02031D502E831620088312A30044
:100C90003E302302031D4F2ECC01CB0AB001A62EFD
:100CA0000D304B02031DA62E0930CB008316200801
:100CB0008312A3002B302302031DA62E83162108C6
:100CC0008312A30043302302031DA62E831622089D
:100CD0008312A3004D302302031DA62E8316230882
:100CE0008312A30047302302031DA62E8316240877
:100CF0008312A30053302302031DA62E0530AA0041
:100D00001D302A020318A52E2A08A03E84000008E0
:100D1000A3004F302302031DA12E2A0AA03E840007
:100D20000008A3004B302302031DA12ECC011E306E
:100D3000CE00D50803199D2ED5030830CB00D9016C
:100D4000A52E0130AA07031C802EB001D508031977
:100D5000C42E0A304B02031DC42EF008031DC42EFE
:100D60000F30D1000230AA002A085502031CBE2E03
:100D70000B30D1070130AA07031CB42ED5260C3046
:100D8000CB000530CD002F100B3057020318282957
:100D90000B305802031828290630590203182C2951
:100DA0000B303002031828293429AA015108AB005E
:100DB0000B302A020318E72E2B080B20AD002A085F
:100DC000313E84002D088000AB0AAA0AD82E080004
:100DD000AA010B302A020318FE2E2A08313E840095
:100DE0000008AD002A083D3E84000008AB002D0835
:100DF0002B020319FC2E0800AA0AE92E5108D6007E
:100E0000080083168C1283128C12181283169816FF
:100E10008312D303AD012D085302031C202F2D088C
:100E2000A03E84000008990083168310981883144C
:100E3000831283181C2F142F0130AD07031C0B2FB6
:100E40004630A400A03084008001840AA40B242F23
:100E50008316981283128C1283168C16831218161E
:100E6000080030304918013EDA003030C918013E20
:100E7000DB0030304919013EDC003030C919013E39
:100E8000DD003030491A013EDE003030C91A013E23
:100E9000DF00080083160512831205120230A50038
:100EA00000301B208316051602308312A500003087
:100EB0001B200800AA0108302A0203187C2F8B137C
:100EC0002D186C2F83160512831205123C301A2040
:100ED000831605168312772F8316051283120512C7
:100EE00000000000831605163C3083121A208B1771
:100EF0000310AD0CAA0A5B2F0800AA0110302A02C9
:100F000003189A2F0310F40CF30CF4178B138316A9
:100F1000051283120512000000008316051600005A
:100F200000008312051A952FF4138B173C301A20FA
:100F3000AA0A7E2FF40CF30CF40CF30CF40CF30C53
:100F4000F40CF30C0F30F4057308E6002B30E400CA
:100F5000E61FB02F2D30E400FF30E606E60AE61368
:100F60003030E5000A306602031CBA2FE50A0A3069
:0E0F7000E602B22F3030E6070800BD2FBE2F7C
:02400E00543F1D
:10420000140014001400140014001400140014000E
:104210003C001900780000003E0001000100380059
:1042200030003900370030003000300030003000FE
:1042300030003000380030003900370030003000E6
:1042400030003000300030003000380030003900DD
:1042500037003000300030003000300030003000D7
:1042600038003000390037003000300030003000B6
:1042700030003000300038003000390037003000A6
:1042800030003000300030003000300038003000A6
:104290003900330030003000300030003000300092
:1042A0003000380030003900370030003000300076
:1042B0003000300030003000380030003900370066
:1042C0003000300030003000300030003000380066
:1042D0003000370033003000300030003000300054
:1042E0003000300038003000390037003000300036
:1042F00030003000300030003000000000000000CE
:00000001FF
